:020000040000FA
:090000000219FD858A6502040A5B
:03000B000215B02B
:0500130002041601FFCC
:0F001B003034F8B283C574C8868BC804C57432FC
:03002B000203E2EB
:03003B000215307B
:03005B0002042577
:10007300C2AF53E67F7592FA7593FFD2AF53917F68
:0C008300302D08C22D303B0302157032F6
:1000B0004A45534330312023323420202020202051
:1000C0000406080C10182030406080A0C0C2AFC0E9
:1000D00082C083901480E493B4541BA3E493B44C83
:1000E00015A3E493B4580FA3A3A3E493B404071295
:1000F0001500D23B8002C23BD083D082D2AF22C255
:10010000AFC2A8C2CAC28EC0D075D008A8CCA9CD33
:10011000D2CAD2AF53E6EF85618BC0E0C0F0758ADA
:1001200000C3E89562F8E99563F9C3E913F9E813A8
:10013000F8E97021E89573401C95735018E582B476
:1001400010137C007B007A007908900000A860C33F
:10015000E813F8215E900000D2A8D2AA6134E0FD35
:10016000C39CC39840EF98EB33FB0582E0FCC39D32
:10017000C39840E198EB33FB0582E0FDC39CC39834
:1001800040D398EB33FB0582E0FCC39DC39840C588
:1001900098EB33FB0582E0FDC39CC39840B798EB16
:1001A00033FB0582E0FCC39DC39840A998EB33FB69
:1001B0000582E0FDC39CC398409B98EB33FB05820E
:1001C000E0FCC39DC398408D98EB33FB058221D999
:1001D000900000D2A8D2AA6134E0FDC39CC398402D
:1001E000EF98EA33FA0582E0FCC39DC39840E1989A
:1001F000EA33FA0582E0FDC39CC39840D398EA3302
:10020000FA0582E0FCC39DC39840C598EA33FA051D
:1002100082E0FDC39CC39840B798EA33FA0582E0B8
:10022000FCC39DC39840A998EA33FA0582E0FDC358
:100230009CC398409B98EA33FA0582E0FCC39DC3B7
:1002400098408D98EA33FA0582EBC46B6A54F0F952
:10025000EAC4303301F454F0C3996009900000D22D
:10026000A8D2AA6134D2C0EBF4C454F0F9EAF4C4C1
:10027000540F49FAEBF4C4540FFBC3EAF99460FA43
:10028000EB9400FB5020C3E97B007A0079006016F4
:10029000C3135006F9C3954D600AE9F54D754E003C
:1002A00079008002054E303A27C3EA94D0F8EB94E7
:1002B00007F9400BE8FAE9FB203109D23141C4309B
:1002C0003102C231203902B231C3EA33FAEB33FBD7
:1002D000EB2B3B3BF9C3EB13FBEA13FAEA29FAEBEE
:1002E0003400FB30E3047AFF7BFFE5255403601BF9
:1002F000202A18E55833F9EB7007C3E99A4002E960
:10030000FAE536C4332AFAEB3400FBC3EA33C454AB
:100310000FF8EB33C454F048F87005EA6002780136
:10032000900000E52260021522614A900000D2A8E8
:10033000D2AA61340522E52270021522C3E5229477
:1003400032500261BF754F0061C2884FD230E86001
:1003500003755000C3E556FC95574002AC57C3ECFB
:10036000954F5008EC75F008A4FAABF0EBF41313BA
:1003700092D5A2E75401F9EAF4FC13A2D513F8E5EB
:100380006423F564EC54032431835564600BE82442
:1003900001E9340020E10208F9C3E89419FAE9946C
:1003A00000FB50047A007B00885189528A538B5499
:1003B00075230A53F7DF43F740800700115577751F
:1003C000230AE5E6A2E082C0400ED2AAD2A8D0F06D
:1003D000D0E0D0D043E6103243E610D0F0D0E0D0E9
:1003E000D032C0D0C0E0C2CF053AE5236002152369
:1003F000C3E54F60057550008105E5502401F550B7
:1004000050037550FFD0E0D0D032C0E0E565856183
:100410008BF0A3D0E032C2AAD28EC2CA85CC62854C
:10042000CD63D2CA3253F7DFC0E0E5F9E5FA30E137
:100430000F8551FB8552FC8553E98554EA53F7BF7C
:10044000D0E0327901801879038014790A8010791C
:100450000F800C791E80087964800479C880007848
:100460001474F0000000D5E0FAD8F6D9F222790130
:10047000801479038010790A800C791E80087964D1
:10048000800479C880007591007594987595FC7505
:100490009104D22D43E680303B0953E67F302D0690
:1004A000121550202DFDD9DE2278FF20282879A1B1
:1004B000E76023E571601F74FF8571F0848539F072
:1004C00030290375F005A4F8C5F0600278FFC3E891
:1004D00095585002A858885722C3E57094E4E571F6
:1004E0009400E55750031481EA046002F557227521
:1004F000E890220559C3E5599408405330EDF4A81B
:10050000BDA9BE755900E9FA79A0E76041EA700615
:10051000E55A6018800CC3E8955A600EE55A5005FC
:10052000600A1480070460FA8002E55AF55AC39500
:100530005F401B7556C0C394044013755680C39426
:1005400004400B755640C39404400375560022E5E1
:10055000562410500274FFF55622743279A687F0A3
:10056000A4C5F0A2F733F558227570007571F0221A
:10057000C2AFC2CAA8CCA9CDAA3A30CF010AD2CA0A
:10058000D2AFC3EA13FAE913F9E813F8853B3E85C5
:100590003C3F883B893C8A3D22C2AFC2CAA8CCA955
:1005A000CDAA3A30CF010AD2CAD2AFAB3BAC3C881D
:1005B0003B893CC3E89BF8E99C202809F9302C03CF
:1005C0000206AC803FAD3D8A3DF9EA9DFA600678AF
:1005D000FF79FF8013AE3EAF3F8B3E8C3FA83BA917
:1005E0003CC3E89EF8E99FF9C3E57113FBE570137E
:1005F000FAE82AF570E93BF57150067570FF7571E0
:10060000FF020651AA70AB71AC70AD717E047F021F
:10061000C3EB9404400D1E1FC3EB94084005202932
:10062000021E1FC3ED13FDEC13FCDEF7C3EA9CFAB8
:10063000EB9DFBEF6009C3E913F9E813F8DFF7EA74
:1006400028FAEB39FB8A708B7150067BFF8B708B1D
:1006500071C3EB94025002D22C3028057F030206AE
:100660007D7892E6FFC3E537948240110FC3E537EA
:1006700094A040010FC3EF940640027F057E02E57F
:1006800071C4540FF9E571C454F0F8E570C4540F07
:1006900028F8C3E89EFAE99400FB4009C3EA9401F4
:1006A000EB940050047A01E4FB0206F8AA70AB71E7
:1006B000EBC4FEEAC4540F4EFCC3EA9CFAEB940070
:1006C000FBC3E813C313F8EA28FAEB3400FB8A7083
:1006D0008B71C3EB94024002C22C7802EBC4FE7B08
:1006E00000EAC4540F4EFAC3EA98FA4005C39401D5
:1006F00050027A017892E6FF303B0953E67F302DB5
:1007000006121550202DFD854992854A93D22D431E
:10071000E680C3E49AF8E49BF9302C03020790E8E2
:10072000FAE9FBD3E913FDE813FC8849894AC3EFD2
:1007300094036038EF20E00CE82CF8E93DF9ECFA7E
:10074000EDFB8013E828F8E939F9C3E82401F8E95A
:100750003400F97AFF7BFFC3EF9403400F8A4B8B81
:100760004C884589468C478D480207C5884B894C83
:100770008A458B468C478D48302812754BF0754C56
:10078000FF7547F07548FF7549F0754AFF0207C5C8
:10079000E8FAD3E813FC8849C3EF94036021EF2003
:1007A000E007E82CF8ECFAE1B0E8282401F87AFF39
:1007B000C3EF940340098A4B88458C470207C588DC
:1007C0004B8A458C47303B0953E67F302D06121586
:1007D00050202DFD753402D22D43E680E5255403CB
:1007E0006034A870A971C3E913F9E813F8C3E913D9
:1007F000F9E813F8302804E92440F9C2AF53E67F42
:10080000759100C3E498F594E499F595759104D237
:100810002D43E680D2AF22D22075440075200030EF
:100820002B03752040800ED2207544007520403087
:100830002B0375200078017901202C20E525540335
:100840006002C2207914E571C313700104F8C394E7
:100850001440027814302804781B791B202D11E5F0
:1008600044600D302803D53404D22101E41207D7A7
:100870000544E59B5440B52004D2A001CCC2A03071
:10088000280908C3E899400118015C20200B08C31F
:10089000E8994003020835015CC22053E67F759158
:1008A00000302C117594007595F8759104D22D4384
:1008B000E680020835E5717EFFC3334005C333404F
:1008C00001FEC3E49E759400F59501AAC3E5339437
:1008D000015003020835302003020835D80201E236
:1008E000015CC221C2A0C2AF53E67F759100854B67
:1008F00094854C95759104854592854693D22D43F8
:10090000E680D2AFE5255403600720290205338035
:100910001030210D202B0A2020071581158102118E
:10092000532278003020027801E53775F007A4F9EA
:10093000E5F028F5F0E9A2F013A2F113A2F213F505
:1009400037C394785003753778C3E5379538400935
:10095000C291C292C29375D57F303B0953E67F3076
:100960002D06121550202DFD854792854893D22DD6
:1009700043E68022203810C2AFC295D29475D53795
:10098000D2AF759F454144C2AFC295D29675D56D21
:10099000D2AF759F454144203810C2AFC29375D580
:1009A0005BD294D2AF759F654144C2AFC29175D5F9
:1009B0005BD296D2AF759F754144203810C2AFC24A
:1009C00094D29675D55BD2AF759F758077C2AFC252
:1009D00096D29475D55BD2AF759F6580672038102D
:1009E000C2AFC29275D56DD296D2AF759F45805475
:1009F000C2AFC29275D537D294D2AF759F458044AD
:100A0000203810C2AFC296D29575D56DD2AF759F02
:100A1000658031C2AFC294D29575D537D2AF759F7C
:100A2000758021203810C2AFC29175D537D295D2CA
:100A3000AF759F75800EC2AFC29375D56DD295D23A
:100A4000AF759F65227A1C7B3C80127A147B4B80A9
:100A50000C7A107B5A80067A0A7B788000E55BD599
:100A6000E001227902E4C295D5E0FDD292D5E0FD05
:100A7000C292D5E0FDD295D5E0FDE920E002D29109
:100A800030E002D293E55BD5E0FDE920E002C291BF
:100A900030E002C2937496D5E0FDD9C9EAF8D5E0FA
:100AA000FDD8FBDBB8C29522C291C292C293C29418
:100AB000C295C29675D57F22788076FF0876FF08AA
:100AC00076FF0876FF0876FF0876FF087609087635
:100AD000FF087601788C76010876FF0876FF0876A5
:100AE000FF0876FF0876FF0876030876FF0876FF92
:100AF0000876FF0876250876D0087628087650080C
:100B000076040876FF0876020876FF08767A08767B
:100B1000FF0876070876010876FF0876FF0876005A
:100B2000087600227888E6C39403D23A5002C23A8B
:100B3000C238E630E102D238A23892397886E6141B
:100B40009000C09378A6F67886E6F539C3940250F3
:100B500003753902789CE67538FFB402037538A036
:100B6000B4030375388278A0E6F860067428240977
:100B7000D8FCF55F2278A5E6F95403D2827002C250
:100B800082E9540C7000E954307000E954C07000E0
:100B900022755D00755E007597DE7597AD7581C035
:100BA00043FF8075EF0675A90075A90051A87580EF
:100BB000FB75F10F75A4047580FB75D4FF7590006B
:100BC00075F27E75A57E75900075D57F75A0007550
:100BD000A601E5B525E0600975A71075CF0075A7DA
:100BE0000075E34075E20251A8E4F8F6D8FD51B86B
:100BF0001211897898865B753001756401C2AF1255
:100C0000045B514512044F12044F12044F514B1212
:100C1000044F12044F12044F515112044F12044F4B
:100C200012044F515751571204577175C2AF53A454
:100C3000F7D283755D00755E00AAE475E4B378FAB7
:100C400079FA308309D9FBD8F7021C008AE4C2AFD5
:100C500071247898865B51A875C804759104C22DDB
:100C600075D84075D90875F781759E03759602751C
:100C7000DA4275DB4275A82175E61043B805759B0D
:100C800080759D0075D10C75BC5975BB1075E880D9
:100C900075B20112044390000075880075720875E2
:100CA0003600C230754D00754E0075E43B1200CD24
:100CB000D2337588517589AA758C00758D00C2A9CB
:100CC000D2ABD2AAD2AF758E017561C075601475B2
:100CD000735075220A1200CD12047E756010C3E5B0
:100CE00022940A754D00754E004077758E0C756123
:100CF0008075602875732875220A1200CD12047E53
:100D0000756020C3E522940A754D00754E0040526F
:100D100075E4B3C233758E017561C0756014757367
:100D20005075220A1200CD12047E756010C3E522B0
:100D3000940A754D00754E004028758E0C756180C3
:100D400075602875732875220A1200CD12047E750D
:100D50006020C3E522940A754D00754E00400302E1
:100D60000C2C120472203003020C2CC2AFA233826E
:100D70003B400651575157800451515151D2AF1247
:100D8000048212047EC3E54F9401400280EFC2AF9B
:100D9000A233823B401D5145D2AF12047EC2AF51F7
:100DA00045D2AF12047EC2AF5145D2AF12047EC20B
:100DB000AF8006515751575157D2AF120482753048
:100DC00000757000757100754000754100E4F531E3
:100DD000F53275200005203001477520000531E50A
:100DE00031F4703D0532789AE67819146012783241
:100DF00014600D787D14600878FA14600375320071
:100E0000C3E53298401B51A81204431532753100D6
:100E10007899865BC2AF5157D2AF7898865B12043F
:100E20007E120476E5237002812C12046E3030A508
:100E3000C3E54F9401500AC3E54D94015016020DCD
:100E4000D512047EE5237003020C2C754D00754EFF
:100E500000020FF4C3E54D94017015C2AF51A8789C
:100E600099865B51457898865BD2AF12047EE1E4A7
:100E7000C3E54D94027015C2AF51A87899865B51B5
:100E80004B7898865BD2AF12047EE1E4C3E54D94C3
:100E9000037015C2AF51A87899865B515178988636
:100EA0005BD2AF12047EE1E4C3E54D94047015C239
:100EB000AF51A87899865B51577898865BD2AF126C
:100EC000047EE1E4C3E54D94057015C2AF51A878E6
:100ED00099865B51577898865BD2AF12047EE1E425
:100EE000C3E54D9407701AC3E54E94065002020EF6
:100EF0002A7401303A0274037888F6C238C239E1A4
:100F0000E4C3E54D9408701AC3E54E9406500202FE
:100F10000E2A7402303A0274047888F6D238D23934
:100F2000E1E4C3E54D94097018C3E54E94065003FF
:100F3000020E2A303A0BC37888E69402F6C23AE1F0
:100F4000E4C3E54D940A7017C3E54E9406500302BE
:100F50000E2A203A0A7888E62402F6D23AE1E4C35F
:100F6000E54D94147026C3E54E94065003020E2AF4
:100F7000C2AF901A0B740093D2AF7888F613C238C0
:100F8000C2394002D2384002D2398058C3E54D946C
:100F9000157038C3E54E94064050C2AF901A0B74DA
:100FA0000093D2AFF8B801027402B802027401B81B
:100FB00003027404B8040274037888F613C238C2BA
:100FC000394002D2384002D2398019C3E54D940C21
:100FD0007012755DA5755EF1C3E54E9406400B1267
:100FE00011D0D2AF754E00754D00755D00755E0075
:100FF000C230C12AC2AF51A8E4D2AFE4F559F524FA
:10100000F525F53775590812046E1204EF30EDFD21
:10101000A8BDA9BEE97001F8885A1204F3755908F1
:10102000C2AF12055A855856855857D2AF303A0785
:10103000C238303102D238D228753300120A001279
:101040000A231205691205991205691205991205FC
:101050006912082712092212097412059912081739
:10106000202C031204A9302C031204D912092212D5
:1010700009971205991208271209221209BA1205B6
:10108000991208171209221209DD12059912082770
:10109000120922120A001205991204EF12081712FF
:1010A0000922120A231204F31205993028278558C1
:1010B0005679187A0CC3E53399400EC228D2298A92
:1010C00035855856855857800CC3E54F9401400329
:1010D000021051215B30291F202B1CE535147006AE
:1010E000C229D22A0151F535203A07C3E54F9401B0
:1010F00040030210518064753600203A0F78FA7967
:10110000A4E760027803C3E55098504FE523604B95
:10111000303A17203805203107800F303102800A1D
:10112000202B07D22B855856018178F0302B05856E
:1011300058567820C3E571985003021051302B1B8C
:10114000C22BC238303102D238D2297535128558B7
:101150005601510536E54F6002215E753600C2AF7B
:10116000120AA8752500D2AF12047E120AA87524AF
:101170000078A4E66006D294D295D296C3E5369460
:10118000044003020C2C020DC1901A0D7820510965
:10119000E520B4550AA35109E520B4AA02801375CD
:1011A0005DA5755EF1120AB831D0755D00755E00FF
:1011B000801D901A0378807B0A5109A308DBFA90FE
:1011C0001A0F788C7B1A5109A308DBFA901A29228E
:1011D000C2AF514C5129901A007402510EA37403EE
:1011E000510EA37421510E901A0378807B0A510D81
:1011F000A308DBFA901A0F788C7B1A510DA308DB39
:10120000FA515F513D901A2922E493F622E6438F6A
:1012100001538FFDFFC3E583941C400122EF855DE0
:10122000B7855EB7F0538FFE22438F02438F01854F
:101230005DB7855EB7901A0DF0538FFC22901A0DA2
:101240007455510E901A0E74AA510E227A3079D02C
:101250007820901A405109E520F709A3DAF7227A9D
:101260003079D0901A40E7510E09A3DAF9227C05B3
:0F12700012045BDCFB22C2AF120A45D2AF22226E
:06148000544C5802030465
:10150000E4F52B757749757816757A10F57BF579C2
:10151000757CD885727D752B00E5E4A2E7B3E5E61E
:0815200092E0F5E60215B42289
:0315300002160B95
:1015500085817685D075E579857AD0857C81D25A6A
:08156000C077C07843E6802249
:10157000305A17C25A85D07AF579D078D0778581DC
:0B1580007C8576818575D085D77B3295
:1015B0000215DE32751CF6751DEB751EE07519BA45
:1015C000751AFEE573751B01B42812751CFC751D98
:1015D000F6751EF1751942751AFF751B0C22C2595A
:1015E000C572F452A4F44280C572C28CC28E758A50
:1015F00000758C007589AA851B8EC289C28BD2AA00
:10160000D2A8C2A9C2BBD28CC23432C2C0C0E030A0
:10161000592AD234E57D428042A4D0E07574A87581
:101620008921538EF0758BFF851A8C85198AC28D9E
:10163000C28FD2BBD28CD28E43A80A32D2AAD2A8F1
:10164000D0E0327B007A0180352059FD2034FA2029
:101650002906202803202000C2AFAB71AA70D2AFA8
:10166000EBC313FBEA13FAEBC313F9EA132AFAE903
:101670003BFBEA24FFEB34FF400474FFFBFAE4FC7D
:10168000C3EB136007FBEA13FA0C80F4EC234B5412
:101690000FC4FBEAC4FA540F4BFBEA54F0FA6BC4D4
:1016A0006B540F4A640FFA78A874E0C0E07416C057
:1016B000E0791C7D17EA540F242B83C0E0C015EAA3
:1016C000C4540F242083C0E0C015EB540F241683AC
:1016D000C0E0C015EBC4540F240B83C0E0C015223A
:1016E0007600D259C149000C1B24303F4B5766721B
:1016F0007C8693A2AFBC0000000000000000000048
:10170000E7F608A61C08A61E08791C22E7F608A61C
:101710001C08A61D08A61C08791C22E7F608A61EB0
:1017200008791D22E7F608A61E08A61C08791C22C7
:10173000E7F608A61C08A61C08A61D08791C22E7C7
:10174000F608A61D08A61D08791C22E7F608A61DA6
:1017500008A61C08791D22E7F608A61D08A61C0885
:10176000A61C08791C22E7F608A61C08A61D087905
:101770001D2209E7F608A61E08791C2209E7F608CB
:10178000A61D08791D2209E7F608A61D08A61C0853
:10179000791C22E7F608A61C08A61C08A61C0879D6
:1017A0001D2209E7F608A61C08A61D08791C2209B7
:1017B000E7F608A61C08A61C08791D2209E7F6080A
:0C17C000A61C08A61C08A61C08791C2208
:1019E0007597DE7597AD43EF02B4A5030219FD901C
:0A19F000FBFDE493B4A5F502FBC073
:1019FD00020B91020321FFFFFFFFFFFF09FF01FF14
:101A0D0055AA01FFFFFFFFFF03FFFFFF25D0285061
:0D1A1D0004FF02FF7AFF0701FFFF0000FF3A
:101A4000234D5F4C5F353023202020202020202094
:101A500023424C48454C492445464D3842313023B9
:101A60002020202020202020202020202020202076
:101C0000C2AFC2D37597DE7597AD7581C075A90057
:101C100075A90043FF80752438752503B1DE752949
:101C2000A5752AF143F10853A4F7D28375D4FF7543
:101C3000E3407DFA780379E67C1075220075230075
:101C4000901DEB7B06752498752501308302814B2E
:101C5000208308D8FBD9F9DCF781BD308308D8FB95
:101C6000D9F9DCF781BDB19EE493A3C39A6004DD8A
:101C7000C381BDDBDBB190600281347B08E493FA61
:101C8000A3B171DBF87A30B171752200752300B110
:101C900090EAFCEBFDC3ED94FE400EB1908A278BD9
:101CA00028ED30E0048A828B83B1907AC270D8C369
:101CB000ED94FE601950CEBD0029EC600F75200038
:101CC0007521FF752900752A000200008100A827F0
:101CD000A9280809D804D90281E0B194EAF281D494
:101CE0000D81A9C3ED94035051EDA2E092007AC595
:101CF000C3E5829400E583941C508C200010438F30
:101D000002438F018529B7852AB7F0300027A8271D
:101D1000A9280809438F01538FFDD804D902A135A2
:101D2000C3E583941C4003A3A11AE28529B7852A41
:101D3000B7F0A3A11A538FFC81857AC1BD030CE4CF
:101D400093A3FAB155DCF8B14D81858187AA22AB06
:101D500023B171EBFAEA6222752608C3E52313F575
:101D600023E52213F52250066323A0632201D52622
:101D7000EAB1DEB1DE75260AEAF4200102D2833030
:101D80000102C283B1DEC3134002C201D526EB2299
:101D9000B194EAFB208302A194308302A1997526B5
:101DA00008AE24AF25C3EF13FFEE13FEB1E2B1DEA0
:101DB000C3EA133083024480FA30E703632201C38D
:101DC000E52313F523E52213F52250066323A063D0
:101DD0002201D526D9E52265236523F52222AE24EA
:101DE000AF250E0FDEFEDFFCD20122424C48656CAF
:091DF0006934373164E8B10601E1
:00000001FF
